:020000040000FA
:1000000001288B138C018316083086008117831218
:1000100086190C288C0A0828831600308600831263
:1000200086110030890083160814831208088D0099
:100030000D1848284B288E0183160830860083123D
:10004000861924288E0A2028831600308600831201
:10005000861103010C080E029100031D30281B2895
:100060009103031D34281B289103031D38281B28E6
:100070009103031D3C281B2883120030890083163E
:100080000814831208088D008D0A0D1848284B2883
:10009000043086004E28023086004E280030890049
:1000A0000D0888008316081555308900AA3089008C
:1000B00088148818592882309400940B60286B2883
:1000C000FF3093000616930B6328FF30930006124F
:1000D000930B68285D28940B6B2882309400940B56
:1000E00072287D28FF3093000616930B7528FF3089
:0C00F00093000612930B7A286F281B283F
:024200000000BC
:00000001FF
